S123E00036373CF6B428C402263EF6A201C50127F9C5802629B6A203847FB7B48A200A3691
S123E020373CF6B428C4022632B7A203F6B428C4032611F6A201C50827F9C5802706BDF8A0
S123E040577EE6D138333239F6A201C501264CF6A209C40127F2B6A20B20BDB7A20BF6A2CE
S123E06009C40827F920C2FEB414C6017FB40081502605C6087CB40081592605C6067CB40A
S123E0800081582605C6047CB40081412602C60381422602C6023AFFB408397FB4287EE62B
S123E0A0D1B7B48916BBB42BB7B42B178D02200444444444840F8B9019894019BDE01FB65C
S123E0C0B48939B6B408BDE0A1B6B409BDE0A139863DBDE01FBDE1A97DB400270DBDE0A1C3
S123E0E0FEB40808FFB408BDE1A9BDE0A139A60027FBBDE01F0820F6BDE0EEBDE17B7FB468
S123E10000CEE174FFB406A6002752B7B4ABBDE01FBDE067BDE0D0B6B4AB814326028D1718
S123E120CEFAC3BDE0EEFEB40608FFB40620D8535848494E5A5643CEFAC5BDE0EECEE12FE1
S123E1408608B7B4ABF6B489862E0C58F7B4892402A600BDE01F087AB4AB26E9398653BD51
S123E160E01F863DBDE01FFCB414C30009FDB408BDE0C33950595841424300860DBDE01F25
S123E180860ABDE01F39B7B40286B78D1E8D1AB1B4022714BDE17BBDE0C3CEFAC8BDE0EEC4
S123E1A0BDE17B8607BDE01F3986B637F6B5FFC4FBF7B5FFB7B421CA02CEE700FFB41FFE5C
S123E1C0B408FFB4228639B7B424B6B402CEB5FFBDB41FF6B5FFC4FDCA04E7003339FEB4A0
S123E1E0143AFFB408398DF6BDE1A9B7B40AFEB40808FFB408BDE1A9B7B40B39CEFFF6FF65
S123E200B4088DE4BDE23C398DD4BDE1A9398DCEB6B40ABDE18639C6088DCBBDE23C39C6AC
S123E220088DBBB6B40ABDE186BDE245B6B40BBDE18639CEB40AFCB408ED0039CEB40AEC5A
S123E24000FDB40839860116FEB4083AFFB408398601B7B4037FB402FCB408B3B402FDB447
S123E2600839FCB40AB3B40826024F39860139CEB4916F00088CB49F26F839CEB491F6B443
S123E280003AEC007CB4007CB400FDB408398608B7B4017FB489CEB491FCB408A3002601B7
S123E2A0390808F6B4895C5CF7B489F1B40123E9395F8608B7B401F7B4008DBF271AF6B5CB
S123E2C0FFCA08F7B5FFBDE1A9F6B40054CEB49F3AA700863FBDE186F6B400F1B40123DA41
S123E2E07EEEE1C6084FF7B400B7B4018D8D270DF6B40054CEB49F3AA600BDE186B6B400BE
S123E3008004B7B400B1B4012AE2394142454B4E5152555B5E6162656B7172757B87C71287
S123E3201314151C1D1E1F08093035383A3C8F8C9CBCCEDEDFFEFF838C8EC3CCCECEE30B52
S123E340A10026057CB405200608BCB4A826F1397FB4167FB42CBDE1A9B7B401CEE31FFFF8
S123E360B4A88DD927567CB405398602B7B4ACBDE37A4AB7B4164C7EE5DEFCB408FDB48BE7
S123E380B6B4AC7DB42C2A014CBDE247CEB49DBDE236BDE250BDE1A9164FFDB40AFCB48B24
S123E3A07DB40B2B0FF3B40AFDB4088602BAB42CB7B42C3970B40BB3B40A20EC16C1CD2611
S123E3C01D8D5281A3270F81AC270B81EE270781EF27037EE47F86C0B7B42C7EE5D5C11A7C
S123E3E026438D3116C4F0C1A02726C1E02722C1B0260E8688C603B7B42CF7B416177EE542
S123E400DDC190260686A0C60220EC8690C60320E6868420F2BDE245BDE1A9B7B401BDE26D
S123E42050B6B40139C11826598680B7B42C8DE5CEE32FFFB4A8CEE327BDE340270B7FB425
S123E44005C681F7B42C7EE5927CB41616C4F0C1A02726C1E02722CEE31FFFB4A8BDE33DF0
S123E460261DC1602713CEE337FFB4A8CEE323BDE340270B7FB4052009BDE2457EE53F7E6C
S123E480E366CEE31FE600F1B4012708088CE32726F32048C40227318604B7B4ABB7B4ACB0
S123E4A0BDE37A8622BDE4AB7EE5D7F6B401C40827028604B7B4AC8603F6B42C2A04CAC0B8
S123E4C02003FAB4ACF7B42C398620BDE4ABC1C027014AB7B4167CB4AB7EE5DDB6B401813E
S123E4E08F275A81CF275684F08170277C81B0277881F02774812026037EE36A8150233D91
S123E500B6B401CEE33DFFB4A8CEE337BDE34027057FB405205A818D2720819D277881AD5D
S123E520271D816E271984F08180274E81C0274A8190275681D0275220447EE36A2070862B
S123E540047DB42C2A0286C0B7B42CBDE245BDE1A936C6047DB42C2A02C606BDE1E6321601
S123E5604FF3B40AFDB4082041F6B42CCA082005F6B42CCA10F7B42C205086102005B6B494
S123E5802C8A04B7B42C8601204DB6B42C8A20B7B42C86012041BDE245BDE1F57FB40ABD02
S123E5A0E23CB6B42C8A20B7B42C7CB41620328601B7B42C7FB416B6B4018139273A813B21
S123E5C0272B813F272286012014B6B40181BD272E817E272A8602BBB416B7B4164CBDE25A
S123E5E047CEB49BBDE23639BDE1FC20F4FEB414C6113ABDE1FF20E9C60ABDE21920E2BD33
S123E600E245BDE1E8BDE23CB6B42C8A08B7B42C8602BBB416B7B41620C7BDE17B863EBDA0
S123E620E01FCC2040B7A202F7A2028601B7A202CEB433BDE000B6B48A811827DD81082641
S123E64008098CB4332DD620EAA700088CB4832704810D26DE860DA7007FB4183981602334
S123E660058020B7B40139373CCEB433F6B4183AA6007CB418B7B40138333986FD5FB7B4DD
S123E680AC4FFDB4128DE0812426028DDABDE65D7CB4ACC6FFF7B42D80302B298109230AE3
S123E6A080078109231F810F221BB7B42DFCB41205050505B7B41217BAB42DB7B4137DB4EA
S123E6C028260220C67CB41739BDE61A201F7CB4058EB5F0BDE17B7DB405270E8607BDE06E
S123E6E01FCEFAA5BDE0EE7FB405BDE61D7FB4177FB404CEFF4FBDE667810D27CC2003BDFF
S123E700E667BDE65D08A60027C4847FB1B401270D7FB4187CB404A6002BE40820F9A60077
S123E7202ADDBDE667810D2719812026E4B6B404810E270E8104270A810F27068D3C810D4F
S123E7402654F6B40458CEE74E3AEE006E00EEEFEAA8E79CE848EB77E8D3EA58E81AE888A9
S123E760F5DFE977F78DEA74E8B6EAC8EED0F6A9F5B5F73BF730F728F6F9BDE67BF6B417E2
S123E78058C10A2211CEB4063AFCB412ED00B6B401812027E5397CB4057EE6D17AB4172B83
S123E7A0467FB4007FB41AFCB408FDB4A8BDE27B2709F6B400C10A26F4202CFCB4A8FDB450
S123E7C008FFB406CEB408F6B41A3A5C5CF7B41AEC00FDB408BDE28E2708FCB408FEB406FE
S123E7E0ED007AB4172AC6BDE17BCEF9F6BDE0EE8673BDE01F863DBDE01F7FB400BDE27B11
S123E8002709BDE0C3CEFAC3BDE0EEF6B400C10823EB7EE6D17CB40520F87AB4172B247F38
S123E820B41ACEB408F6B41A3A5C5CF7B41AEC00FDB408BDE28E26DD6F006F017AB4172ADE
S123E840E120A4BDE26F209F7AB4172B132657BDE233C608BDE20EBDE245B6B40BBDE18678
S123E860BDE217BDE28E27037EE2B17CB427F6B5FFCA10F7B5FFBDE217BDE3507DB40526EE
S123E88025C60A860C7EE2B4F6B4175A2B232616FCB408FDB41D270EBDE217CEB429BDE279
S123E8A036BDE28E27C57CB4054F5FFDB41D7EE6D1CC000120DDF6B4175A2B0C26E8FCB445
S123E8C008FDB41B27E020A6CC000120F47CB4057EE6D17FB4A8F6B4175A2BF15A27052A86
S123E8E0ECBDE233B6B40984F0B7B4097DB4A826DF7FB4187FB419BDE17BBDE0C3CEFAC382
S123E900BDE0EEF6A201C401271AB6A203847F8117260AF6A201C40127F9B6A2038118260B
S123E920037EE6D1BDE1A94D2B0881202504817F2502862ECEB433F6B4183AA7007CB4188F
S123E940BDE1A9BDE0A18620BDE01FBDE26226037CB4A8BDE2457CB419F6B419C41027A33C
S123E960CEFAC4BDE0EECEB433A600BDE01F088CB44223F57EE8ECCEFA06BDE17BBDE0F8F5
S123E9807EE6D1F6B404C10C2607F6B419C1062703BDE0D0BDE61DBDE67B7AB4182740CE1C
S123E9A0EA53A600274C08B1B40126F6B6B413F6B404C10C2615F6B419C106260EFCB412C0
S123E9C0830009FDB48DBDE9F92014BDE1867DB400270CBDE250B6B412BDE186BDE245B6E5
S123E9E0B401813D2763815E273D810D2748812E27037CB405B6B401397FB48FFEB4147C20
S123EA00B48FF6B48F3AFFB408BDE1A9FEB48DF6B48F3AFFB408BDE186F6B48FC10926DCA4
S123EA20FEB48DFFB41439BDE2507AB4192AC6C606F7B41920BFBDE245F6B4195CF7B41937
S123EA40C1062FB17FB41920AC7DB40027A7BDE25020A25E3D2E0D007AB41726627FB4006D
S123EA60BDE17BBDE0C3BDE9837DB4052654812E26EE204EF6B4172646C606F7B419BDE1B4
S123EA807BCEE174F6B4193AA6002714BDE067BDE01FBDE9837DB4052628812E272420DE91
S123EAA0BDE15DBDE98320EDF6B417C1032610B6B40DBDE186BDE2622708BDE24520F07C2B
S123EAC0B4057EE6D17EE6D1C601B6B401810D2704BDE66716F7B401BDE17BCEA2008D1E24
S123EAE0E601C50127F8C5802625A60316847FB1B40127D1A609840827FAE70B20E0E60959
S123EB00C401270AA60BA703E601C40827FA398665B7A20A86647FA203F6A201C40827F9B2
S123EB204A26F38675B7A20A8655B7A202BDF85720AC7CB4057EE6D1B6B401810D27F38104
S123EB402026EFBDE667BDE65D8154260AF6B428CA01F7B428200C814826D7F6B428CA026D
S123EB60F7B428397CB418BDE667810D2705BDE01F20F4BDE17B39BDE17BBDEB38F6B4288C
S123EB80C4012603BDEB647FB416BDE000B6B48A815326F6BDE000B6B48A81392706813183
S123EBA026E820037CB4167FB42B8D3A8003B7B4198D33B7B4088D2EB7B4097AB4192B0AD0
S123EBC08D24BDE186BDE24520F1F6B42BF7B4198D147DB416260943B1B41927AD7CB405ED
S123EBE07FB4287EE6D17FB4138D0C8D0ABBB42BB7B42BB6B41339BDE000B6B48ABDE68D64
S123EC007DB42D2BD839CEB429BDE236398DF7CC2032CEB4333AA7005A26F7BDE17B7FB4A2
S123EC2018B6B408BDEE51B6B409BDEE517FB4ABBDE350BDEE44B6B416B7B402B7B4177C33
S123EC40B418BDEE4E7CB418BDE2457AB4022AF2BDEE447DB4052712BDE2507DB42C2A039C
S123EC60BDE2507FB416C64220377FB4077DB42C2A09BDE1A9B7B407BDE245BDE1A9B7B4E0
S123EC800616C40F815F2223165454C10727147DB42C2A0B81352607C68E7CB4052069C64E
S123ECA0FF206516C403CEEE8F205A817F2205CEEE93205181BF2233CEEEA3C103260E7CDB
S123ECC0B405B6B407811A253CC6122038C10C260DB6B407272F81CD272BC6132027818F43
S123ECE026235C7DB42C2A1D5C201ACEEEB781CF2604C612200FC10E250BB6B4072706811F
S123ED00CD27025C5C3AE600F7B4047FB4025FCEF3013AA600810F22035C20F3840FB7B41A
S123ED2019B6B402B1B4042728B6B42C818127034D2B197DB4052614CEF3F417F6B4023A1D
S123ED4016A600CEF3013AB1B40627057CB40220C8B6B42C8181260BB6B404818E27015C7C
S123ED607FB416B6B402B7B404A600840FB1B419221ECEF20E3AA600847FF7B400F6B41955
S123ED80CB16CEB4333AA7007AB4192B0DF6B4005ACEF3013A20CC7EEE2CC61CF7B418B69A
S123EDA0B42C810225F126097FB416BDEE827EEE2CBDE245F6B42CC41027058623BDEE6922
S123EDC07DB4162710BDEE7DBDE1F57AB4162B5C8D7FBDE245F6B42CC538270E7DB4AB2631
S123EDE009C58027E37AB41620DEC544272C862C8D778658C54027114C36B6B406811C2792
S123EE0004811D26037AB416328D5EC4BBF7B42C2A087AB4AB27037AB416B6B4162F0D3601
S123EE208D5732C40227A14A269E8D585FCEB4333AA600BDE01F5CC12D23F2CEB49BBDE26C
S123EE40727FB405CEB429BDE23F39BDE245BDE1A9B7B4018D07B6B401840F200444444429
S123EE60448B30813923028B07CEB43337F6B4183AA7005CF7B4183339862C8DEC86248DA2
S123EE80E8398DF9B6B49B8DC8B6B49C8DC339261325245C00003357006D0E0A6A3A004508
S123EEA0884B2E7F31738108194D7840036005374C507C9091363880327407091A4E7941E5
S123EEC00461064F7A517D527E7B7CB4057EE6D1CEFAD4BDE17BBDE0EE088CFF4F23F4201E
S123EEE0ECBEB414F6B5FFC47FCA01F7B5FF3B7AB41726517FB42FBDEC0D7FB4167FB405A9
S123EF007FB42CBDE61DBDE667810D2609B6B4174CBDE24720E1812E27357AB4187FB419B6
S123EF207FB4047FB430C6FFBDE667BDE65D5CCEF3013AA600810F2305840F7CB404B1B482
S123EF4019270F22E98607BDE01F7FB40520A87EE6D1CEF20E3AF7B489A60027E8847FB130
S123EF60B40126CAA6002B057CB41920BBCEF3013AA60044444444B7B4008104262BBDE658
S123EF8067BDE65D812026057AB418201C814127128142270A8144270220AA5C7CB4045C25
S123EFA07CB4045C7CB40420C4F6B4045ACEF3F43AA600B7B404BDE667812E2704810D2601
S123EFC011B6B4004A27068108270220097AB4182007812027037EEF45F6B40058CEEFE3D4
S123EFE03AEE006E00F183F0BDF080F0BDF17EF0C7F0C7EFFAF1E57EEF4518CEB4ADBDE106
S123F000A9B7B484BDE67B7DB4122668BDF119260D7CB418B6B4048A0CB7B40420037AB45F
S123F02018B6B4048D338D2EBDE67B7DB41226448D24F6B489C1412715C11E2711BDE67BA9
S123F0404FBDF0947DB405262BBDE2508D087CB4308D0F7EF186B6B41318A7001808BDE225
S123F0604539BDE250180918A600BDE186188CB4AD26EF39BDEE44B6B484BDE1867EEFF764
S123F0807CB416BDE67BBDF0917DB40526EF7EF186B6B4164CBDE247FCB412B3B408240D76
S123F0A081FF27037CB4055D2B0F7CB4054D27037CB4055D2A037CB405F7B41339B6B404D1
S123F0C08010B7B404200ABDE667812327487AB4187CB416BDE67B86107DB4AC2F0E7CB45C
S123F0E016F6B400C104260280108B20BBB404B7B404B6B401812C27037EF186BDF119261E
S123F1007DF6B400C104277BB6B4048B10B7B404BDE6677EF1997EF1F1BDE667BDE65D81E8
S123F1205826127DB41227037EEFF78D1B2604861A20394F39815926207DB41226EA861806
S123F1408D18262886CD2024F6B489C159270AC15B2706C1892702C1CD39F6B489C15A27AB
S123F1600AC1882706C1CC2702C1593936BDEE4432BDE186BDE2458680B7B42C4F3920243A
S123F1807AB42FBDE667F6B4898DC427088DDA2608861A200286188DD3B6B401810D2707D5
S123F1A0812E27DC7EEF457DB4302628BDEE447DB42C2A03BDE245B6B404BDE1867DB40513
S123F1C02620BDE245CEB4127AB4162B07260108A60020E6BDEE44BDEC0D7DB42F26037E70
S123F1E0EF0D7EE6D18618BDE1868680B7B42C2092BDE67BF6B400C80727057DB41226A4F9
S123F2007AB4187CB4165D26037CB41620E14142C1D8D94443C1C244C1C2C44E44C1C2539F
S123F220CCC1C2C4D2C1C24243C3D34CD245D147C5D448C9D34954C1C24CC5CFD3D44DC992
S123F2404EC550CC52C1CE434CD25345D45345D4D256C3D34342C14CC3C9D6D2C1C24D50BD
S123F260C1C24FCDC1C250C4D8D94441C145C3C1C2D3D8D9454F52C1C24643C24449D649EE
S123F2804449D64EC3C1C2D3D8D94A4DD053D24C4441C1C2C4D3D8D953CCC1C2C4D2C1C20C
S123F2A0C44D55CC4E45C7C1C24FD04F5241C1C2505348C1C2D8D9554CC1C2D8D9524FCC56
S123F2C0C1C2D2C1C254C9D35342C143C1C245C3C9D65441C1C2C44FD0D3D8D95542C1C206
S123F2E0C457C95441C2D042C14553D450C153D4C1C2D8D958D359D35741C9584744D8D9D8
S123F300000001121292010263630263637301026363014213131342131300013232028397
S123F32001320132320132320102636301323232320132013201320132320203840203842A
S123F34001028332013232000112011212124213130102636301421313017272720001123E
S123F3600142131312129200010263630001520102130001021301421313121292000142C0
S123F38001220001026363727272720142131313421313130001120001421313011200012E
S123F3A0026363000102131313930102131313930001421313421313011212000112026375
S123F3C063011212120102232322021322222201026363730112000112120112010213010B
S123F3E012014213131292011201920001120001021393001B3A3A89C98BCBC384C4684896
S123F4005805674757242515272C2E222485C52F25232D2B262A20211312148D2829110C83
S123F4200E0A6F4F5F81C1634353838C8C196A4A5A34090988C84103026C4C5C3108086EF7
S123F4409D86C6CC8ECECE68485805644454043D604050018ACA36373C3C323338386949CE
S123F460596646563B391082C20D0F0B97D7DDCF9FDFDF80C0833F16061700076D4D5D3044
S123F4803035353E8F8FCE10006F351C3C20CE00E28D198D22A700088C00E726F4164D2BA9
S123F4A01F271D4A276A4A27767E00A7F6102EC42027F9B6102F397D102E2AFBB7102F3989
S123F4C0FE00E286FFA1002609BC00E427030820F24A8DE35D2B0881FE270D8DCF27098DF9
S123F4E0CB8D29FEBFFE6E00FE00E28DBF8DC85F8C103F2602A7008CD0002504C630200237
S123F500CA128D5ABC00E427050820DF20478D9CFE00E2A6008DA0BC00E427C30820F45F09
S123F520FE00E286FFA700CA068D332093FE00E28C103F260486FFA7005FCA168D2008BCB7
S123F54000E42FF520E55CF7103B8D09C620F7103B5FF7103B18CE0C00180926FC39F71028
S123F5603BA7008DE15A39CEB408F7B40CA600BDF4B7BDF4AC088CB40D26F2397CB4057E9F
S123F580E6D18622B7102B860CB7102D86FFBDF4B701CEF486A600BDF4B7BDF690088CF580
S123F5A08523F2CEFFFF0926FD860CB7102DB6102EB6102F39BDF6C48DC8C6FF8D1781FE59
S123F5C02709CEFA0DBDE17BBDE0EEBDF4B78D087F102D20AABDF567BDF555BDF4AC39BD88
S123F5E0F6C4BDF5825F8DED81FE271CCEFA0DBDE17BBDE0EECEFA4BBDE0EEBDE000B6B460
S123F6008A800DBDF4B726C3FEB4083CBDE17BCEFA49BDE0EEBDE0C3BDE1A97DB48D270344
S123F620B6B40DBDF4B7BDF4ACBDF555FEB408BCB40A2705BDE24520D6BDF5AEBDF4B73849
S123F6407FB4A6FFB4087DB48D27037CB48E8D40188C00002606CEFA757EF5C57DB4A6275C
S123F66005BDE186201036BDE1A97DB48E2703B6B40D3310262DFEB408BCB40A2705BDE2BB
S123F6804520CBCEFA677DB4A626CECEFA3920C918CE0680F6102EC4202604180926F5B6B2
S123F6A0102F39CEFA207EF5C58D197FB4A6BDF582C601BDF5677DB48D2703BDF77AFEB453
S123F6C0087EF64E7FB48D7FB48EB6B417270E8102251F220FFCB40AB3B40824067CB405A5
S123F6E07EE6D1397AB417FCB40CFDB40E7CB48D20E3FCB408FDB40A39B6B417810122DD6A
S123F7004A2617FCB4081A83103F2703CCFFFFFDB40ABDF582C6027EF5BCCCB600FDB408A5
S123F720CCB7FFFDB40A20EA8D9A7CB4A67EF6AEBDF6C4BDF582C6037EF5BC7AB417261F32
S123F740CEF765EC0027181AB3B4122704080820F28F83F76554BDF8C7F7A2097EE6D17CDF
S123F760B4057EE6D1015003000600120020002400480018009600019200FCB40AB3B40835
S123F780F3B40EFDB40AFCB40EFDB40839BDF6C4FEB4087DB48D2706FCB40CFDB408EC00C8
S123F7A03CBDE186BDE24538BCB40A27030820EE7EE6D18EB5F0CE00F6FFB41486D0A7011E
S123F7C0C604F7B5FF7FB4287FB400BDE26FBDF7D3202BCEA200CC2238A702A70AE702E782
S123F7E00ACC4010A702A70AE7028601A702CC9317A700E700A708E7088603A70E39CCB0D7
S123F80000ED04CCFFFFED0618CEA20ECEA20DA600840426FA18A600A600840427FA18A60A
S123F82001FEA2065F18CEF9CD183A188CF9DF22CDCDAC0025045C5C20EBBDF8C3F7B4319C
S123F840F7B432F7A2013733F7A2098605B7A202B7A20A8D02203DCEA2008602A70FCC2052
S123F86001A7021C0080E702C604A601850427FAE703A601850127FAA6035A26EDCC2001FF
S123F880A7021D0080E70218CEFFFF180926FC8602A70E39CEF9E1BDE17BF6B428C4FDF74D
S123F8A0B4287FB4057FB427C604F7B5FF4F5FFDB41DFDB4A6FDB41BF6B5FFCA04F7B5FF9F
S123F8C07EE97D5D270154CB03F7B4AC58585858FAB4AC397EF988F6B5FFC4FEF7B5FFBF7A
S123F8E0B414BFB48D8EB5F0BDE217BDE250BDE233860CBDE290270FBDE1A9813F27D5F6A2
S123F900B5FFCA20F7B5FFF6B5FFC4102715C60C860ABDE2E6CEB49BBDE272F6B5FFC4F766
S123F920F7B5FFF6B5FFC4082703BDE2E3BDE21FBDE23CF6B5FFC4202633C604F7B5FFBD44
S123F940E28E2662FCB41D8300012516FCB429B3B4082609FCB41D830001FDB41DFCB41DBC
S123F9602641CEF9F6BDE17B201C7EF89ABDF7D3F6B431E701F6B432E7098605A702A70AFF
S123F980CEF9FEBDE17B20E2FCB414830009FDB48DBDE9F9BDE1FCBDE21F7EEEE17FB42757
S123F9A07EE2B17EE86B7DB42726F2BDEC0DCEFF4FFCB41B830001FDB41B260220ACBDE073
S123F9C0FB7EE86ECEFA83BDE0EE7EE6D1FA02FD02FE82FF42FF8FFFA2FFD20000FFEDFFA2
S123F9E0F60D0A202045564D62756731312052657620322E3500202042726B7074002020A9
S123FA0041626F727400202052656773004D43363848433131204E4F5420424C414E4B0095
S123FA204D4336384843313120444F4553204E4F5420564552494659005645524946592091
S123FA40434F4D504C455445000D000D0A454E5445522052455455524E20544F20434F4EE4
S123FA6054494E554500005245414420434F4D504C455445004552524F5220494E20524570
S123FA80414400494E54455252555054204F4343555252454420494E204D4F4E49544F529A
S123FAA0204D41500020494C4C4547414C2F494E53554646494349454E5420454E545259C2
S123FAC00D0A00202020200020424144204D454D4F525900425245414B203D2041626F7245
S123FAE07420636F6D6D616E642C204354524C2D41203D2045786974207472616E73706170
S123FB0072656E74206D6F64652C204354524C2D48203D204261636B73706163652C200027
S123FB204354524C2D57203D20467265657A652073637265656E2C204354524C2D58203D27
S123FB402043616E63656C20636F6D6D616E64206C696E650041534D203C53544152542089
S123FB60414444523E2D2053696E676C65206C696E6520617373656D626C65722F64697364
S123FB80617373656D626C6572004246203C535441525420414444523E203C454E44204124
S123FBA04444523E203C444154413E2D20426C6F636B2066696C6C206D656D6F727900427B
S123FBC052205B3C4144445231202D2041444452353E5D2D20536574203120746F20352032
S123FBE0627265616B706F696E74730042554C4B205B3C313033463E5D2D2042756C6B200A
S123FC00657261736520736C617665204D435520454550524F4D206F7220434F4E464947D1
S123FC20004348434B203C535441525420414444523E205B3C454E4420414444523E5D2DB3
S123FC4020426C616E6B20636865636B20736C617665204D435520454550524F4D2E2042C2
S123FC606C616E6B2062797465203D20464600434F5059203C535441525420414444523E5F
S123FC80205B3C454E4420414444523E203C555352204D41502053544152543E5D2D434FFD
S123FCA0505920736C617665204D435520454550524F4D20746F2055736572204D6170452A
S123FCC052415345203C535441525420414444523E205B3C454E4420414444523E5D2D20E1
S123FCE04279746520657261736520736C617665204D435520454550524F4D0047205B3C16
S123FD00535441525420414444523E5D2D20476F20746F2075736572206D617020616E64E5
S123FD2020657865637574652070726F6772616D004C4F4144203C504F52543E205B3D3CA1
S123FD40544558543E5D2D20446F776E6C6F6164202848296F7374206F722028542965728E
S123FD606D696E616C20706F727420746F2075736572206D6170004D44203C5354415254CE
S123FD8020414444523E205B3C454E4420414444523E5D2D204D656D6F72792064697370EC
S123FDA06C6179004D4D203C414444524553533E2D204D656D6F7279206D6F646966790051
S123FDC04E4F4252205B3C4144445231202D2041444452353E5D2D2052656D6F7665206256
S123FDE07265616B706F696E74730050205B3C434F554E543E5D2D2050726F636565642065
S123FE00312D464646462074696D6573207468726F756768206120627265616B706F696EA9
S123FE20740050524F47203C535441525420414444523E205B3C454E4420414444523E2088
S123FE403C444154413E5D2D50726F6772616D20736C617665204D435520454550524F4D80
S123FE600052442D20526567697374657220646973706C617900524D2D20526567697374E6
S123FE806572206D6F64696679005350454544203C4241554420524154453E2D2053656CFB
S123FEA065637420686F7374206261756420726174650054205B3C434F554E543E5D2D2020
S123FEC0547261636520312D4646464620696E737472756374696F6E7300544D205B3C45A7
S123FEE0584954204348415241435445523E5D2D205472616E73706172656E74206D6F6482
S123FF00650056455246203C535441525420414444523E205B3C454E4420414444523E20BB
S123FF203C555352204D41503E5D2D2056657269667920736C617665204D435520454550F2
S123FF40524F4D20746F2075736572206D6170004153CD42C642D2C74C4F41C44DC44DCD60
S123FF604E4F42D2D050524FC752C4524541C452CDD454CD48454CD0564552C6434843CB89
S116FF8053504545C445524153C5434F50D942554CCB0020
S123FFD6F9C4F9C4F9C4F9C4F9C4F9C4F9C4F9C4F9C4F9C4F9C4F9C4F9C4F9C4F9C4F9C437
S10DFFF6F8D7F7B3F9C4F9C4F7B360
S9030000FC
